:10000000C128A501A400B3172730A3001030142085
:100010000330A300E8301420A30164301420A301AE
:100020000A30142024081F28A2002508A100240853
:10003000A000A0202008031DB313B31B0800303E0E
:10004000A600360884000930A70003102C20A60C57
:10005000A70B262803142C288413B31D3B28000863
:100060003404331D34068000841700083404031C54
:1000700034068000462800083404031C3406331973
:10008000340680008417340980054628330D06396C
:10009000A0004F20A100A00A4F20000091280030AE
:1000A0008A0020088207013499340334393400343B
:1000B00060340C34FD346400712003185B287C200C
:1000C000A8010830A3007D2071200318A80AAB1EE8
:1000D000A801A20CA30B6328AB1AA2137D2022084F
:1000E000080036088400340884178004841300054F
:1000F0002B1B3406FF3E080033172B081F39003E28
:10010000A1002A080E3E0318A10A331F91283313B9
:10011000A0000310A10CA00C0310A10C200C91282E
:10012000A101FC3EA000A109031C9C28FF30000097
:10013000A00703189728A0076400A10F96280800BD
:10014000A501A4011030A600210DA40DA50D2208C3
:10015000A4022308031C230FA5020318B6282208B3
:10016000A40723080318230FA5070310A00DA10D52
:10017000A60BA4282008BC28831303138312640051
:10018000080083168501860181308700880183126B
:100190000716831607128312881783168813831293
:1001A0000817831608138312881683168812831281
:1001B0000816831608128312881583168811831275
:1001C0000815831608118312881483168810831269
:1001D0000814831608108312861783168613831259
:1001E0000617831606138312861683168612831249
:1001F000061683160612831286158316861183123D
:100200000615831606118312861483168610831230
:10021000061483160610831209158316091183121A
:100220008914831689108312091483160910831206
:100230008516831685128312851583168511831200
:1002400005158316051183128514831685108312F4
:1002500005148316051083120730B6008030B400F1
:100260000C30AA00AB018A015B20B8008A015B2038
:10027000B9008A015B20BA00103087068316071286
:1002800007308312B6002030B4000630B3003808BF
:100290008A01012020308A01202039088A010120AA
:1002A00020308A0120203A088A0101200A308A0180
:1002B00020200D308A01202064003808903C8A11EB
:1002C0000A120319742A64003808803C8A110A1241
:1002D00003196A29640039083C3C8A110A12031D7B
:1002E00075298817831688138312640039083D3CEA
:1002F0008A110A12031D8029081783160813831216
:10030000640039083E3C8A110A12031D8B298816A5
:10031000831688128312640039083F3C8A110A123E
:10032000031D9629081683160812831264003908E3
:10033000403C8A110A12031DA129881583168811D1
:10034000831264003908413C8A110A12031DAC294A
:10035000081583160811831264003908423C8A117B
:100360000A12031DB72988148316881083126400AB
:100370003908433C8A110A12031DC2290814831646
:100380000810831264003908443C8A110A12031DC4
:10039000CD29861783168613831264003908453CDD
:1003A0008A110A12031DD829061783160613831211
:1003B00064003908463C8A110A12031DE329861697
:1003C00083168612831264003908473C8A110A1288
:1003D000031DEE29061683160612831264003908DF
:1003E000483C8A110A12031DF929861583168611C5
:1003F000831264003908493C8A110A12031D042A39
:100400000615831606118312640039084A3C8A11C6
:100410000A12031D0F2A86148316861083126400A5
:1004200039084B3C8A110A12031D1A2A0614831636
:1004300006108312640039084C3C8A110A12031D0D
:10044000252A0915831609118312640039084D3CC9
:100450008A110A12031D302A891483168910831207
:10046000640039084E3C8A110A12031D3B2A091404
:10047000831609108312640039084F3C8A110A124E
:10048000031D462A851683168512831264003908D7
:10049000503C8A110A12031D512A851583168511B5
:1004A000831264003908513C8A110A12031D5C2A28
:1004B000051583160511831264003908523C8A1110
:1004C0000A12031D672A851483168510831264009F
:1004D0003908533C8A110A12031D722A0514831627
:1004E000051083128A012C29640039083C3C8A11CA
:1004F0000A12031D7F2A881383168813831264004F
:1005000039083D3C8A110A12031D8A2A08138316F2
:1005100008138312640039083E3C8A110A12031D35
:10052000952A8812831688128312640039083F3C8A
:100530008A110A12031DA02A0812831608128312B8
:1005400064003908403C8A110A12031DAB2A881145
:1005500083168811831264003908413C8A110A12FB
:10056000031DB62A08118316081183126400390886
:10057000423C8A110A12031DC12A88108316881072
:10058000831264003908433C8A110A12031DCC2AE5
:10059000081083160810831264003908443C8A113D
:1005A0000A12031DD72A861383168613831264004A
:1005B0003908453C8A110A12031DE22A06138316E4
:1005C0000613831264003908463C8A110A12031D7F
:1005D000ED2A861283168612831264003908473C7E
:1005E0008A110A12031DF82A0612831606128312B4
:1005F00064003908483C8A110A12031D032B861136
:1006000083168611831264003908493C8A110A1244
:10061000031D0E2B06118316061183126400390880
:100620004A3C8A110A12031D192B86108316861064
:100630008312640039084B3C8A110A12031D242BD3
:100640000610831606108312640039084C3C8A1188
:100650000A12031D2F2B091183160911831264003E
:1006600039084D3C8A110A12031D3A2B8910831652
:1006700089108312640039084E3C8A110A12031D46
:10068000452B0910831609108312640039084F3C6A
:100690008A110A12031D502B8512831685128312AC
:1006A00064003908503C8A110A12031D5B2B851126
:1006B00083168511831264003908513C8A110A128D
:1006C000031D662B0511831605118312640039087A
:1006D000523C8A110A12031D712B85108316851056
:1006E000831264003908533C8A110A12031D7C2BC3
:1006F00005108316051083128A012C2963008A01D4
:020700007E2B4E
:02400E00763FFB
:00000001FF
